:020000040800F2
:10000000201100200D0C000825030008270300081C
:100010002B0300082F030008330300080000000032
:10002000000000000000000000000000370300088E
:1000300039030008000000003B0300083D030008EE
:10004000270C0008270C0008270C0008270C0008C4
:10005000270C0008270C0008270C0008270C0008B4
:10006000270C0008270C0008270C0008270C0008A4
:10007000270C0008270C0008270C0008270C000894
:10008000270C0008270C0008270C0008270C000884
:10009000270C0008270C0008270C0008270C000874
:1000A000270C0008270C0008270C0008270C000864
:1000B000270C0008270C0008270C0008270C000854
:1000C000270C0008270C0008270C0008270C000844
:1000D000270C0008830B0008270C0008270C0008D9
:1000E000270C0008270C0008270C0008270C000824
:1000F000270C0008270C0008270C0008270C000814
:10010000270C0008270C0008270C0008270C000803
:10011000270C0008270C0008270C0008270C0008F3
:10012000270C0008270C0008270C0008270C0008E3
:1001300000F002F800F05EF80AA090E8000C82449B
:100140008344AAF10107DA4501D100F053F8AFF278
:10015000090EBAE80F0013F0010F18BFFB1A43F0A5
:1001600001031847541F0000741F000010F8013BE2
:100170000A4413F0030408BF10F8014B1D1108BF17
:1001800010F8015B641E05D010F8016B641E01F8C5
:10019000016BF9D1002D15D010F8014B03F00C03C1
:1001A0000C2BA1EB04040ABF10F8013BA4EB831451
:1001B000A4EB032405F1010314F8016B5B1E01F8A5
:1001C000016BF9D5914238BF10F8013BD1D370478C
:1001D0000023002400250026103A28BF78C1FBD850
:1001E000520728BF30C148BF0B6070471FB51FBD05
:1001F00010B510BD01F021FB1146FFF7F7FF00F02D
:1002000009F801F03FFB03B4FFF7F2FF03BC00F075
:100210005DFC000008B500F0E9FB00F051FC00F0C7
:1002200012FB00F0E7F9202467E000F0E3F9002278
:100230001146104600F09BFA01220021122000F026
:1002400096FA02220021242000F091FA03220021D4
:10025000362000F08CFA04220021482000F087FAB2
:10026000052200215A2000F082FA062200216C208B
:1002700000F07DFA21A20321002000F05DFA23A204
:100280000621002000F058FA22A206213F2000F0AB
:1002900053FA22460621302000F0CCF9601CC4B28B
:1002A0007E2C00DD2024102003232246062100900E
:1002B000672000F0FFF94FF4FA5000F0D4FB00F093
:1002C00099F94FF4FA5000F0CEFB1448082380222D
:1002D00000210090084600F07BFA4FF4FA5000F03D
:1002E000C2FB0F480823802200210090084600F03E
:1002F0006FFA4FF4FA5000F0B6FB96E7312E332731
:10030000204F4C4544205445535400004153434929
:10031000493A0000434F44453A00000000000020E5
:1003200000040020704700BFFEE700BFFEE700BFEB
:10033000FEE700BFFEE77047704770477047000058
:100340000CB50020019000906C48006840F48030AB
:100350006A49086000BF6948006800F400300090F6
:100360000198401C0190009818B90198B0F5A06F51
:10037000F1D16248006800F4003010B10120009013
:1003800001E0002000900098012843D15C480068FB
:1003900040F010005A4908600846006820F0030049
:1003A00008600846006840F0020008605348406852
:1003B000524948600846406848600846406840F432
:1003C000806048600846406820F47C104860084619
:1003D000406840F4E81048600846006840F08070CB
:1003E000086000BF4548006800F000700028F9D0A0
:1003F0004248406820F00300404948600846406891
:1004000040F00200486000BF3C48406800F00C002B
:100410000828F9D10CBD10B5FFF792FF10BD10B53B
:100420003648006840F001003449086008464068DA
:10043000344908403149486008460068324908405C
:100440002E4908600846006820F4802008600846AD
:10045000406820F4FE0048604FF41F008860FFF7FA
:10046000DAFF4FF000602949086010BD10B5002187
:1004700000200022214B5B6803F00C0121B104290C
:1004800006D0082928D107E0214B224C236027E021
:100490001F4B204C236023E0184B5B6803F4701063
:1004A000164B5B6803F48032022303EB904022B9C1
:1004B000194B4343174C23600DE0104B5B6803F46A
:1004C000003323B1144B4343124C236003E0104B21
:1004D0004343104C236003E00D4B0E4C236000BFE0
:1004E00000BF064B5B68C3F303130C4CE15C094B84
:1004F0001B68CB40074C236010BD00000010024079
:10050000002002400000FFF8FFFFF6FE08ED00E0CB
:1005100000127A000008002000093D0004080020B5
:1005200070B504460E4626B14021FE4800F009FD94
:1005300003E04021FB4800F006FD1021F94800F0DF
:1005400002FD002517E02021F64800F0FCFC04F035
:10055000800020B18021F34800F0F3FC03E080210B
:10056000F04800F0F0FC2021EE4800F0EAFC6006C4
:10057000040E681CC5B2082DE5DB1021E94800F027
:10058000E0FC4021E74800F0DCFC70BD70B504469B
:100590000D4605F1B001C8B20021FFF7C1FFA11C53
:1005A000C1F3031141F010000021FFF7B9FFA11CB6
:1005B00001F00F000021FFF7B3FF70BD10B500215F
:1005C0008D20FFF7ADFF00211420FFF7A9FF0021C8
:1005D000AF20FFF7A5FF10BD10B500218D20FFF75C
:1005E0009FFF00211020FFF79BFF0021AE20FFF7A7
:1005F00097FF10BD70B5002419E004F1B001C8B236
:100600000021FFF78DFF00210220FFF789FF002165
:100610001020FFF785FF002505E001210020FFF7EE
:100620007FFF681CC5B2802DF7DB601CC4B2082CAC
:10063000E3DB70BD2DE9F04107460E4690460025EC
:100640000024A8F12000C5B27F2F02DD0027B01CD6
:10065000C6B231463846FFF799FF002408E004EBA4
:100660000511B14A505C0121FFF75AFF601CC4B26A
:10067000082CF4DB701CC1B23846FFF787FF00245A
:1006800009E004EB05110831A74A505C0121FFF78E
:1006900047FF601CC4B2082CF3DBBDE8F08110B545
:1006A0000246012000E050430B1EA1F10104E1B21B
:1006B000F9D110BD2DE9FF5F074691461D460E9EFC
:1006C0004FF0000A002433E0281B401EC1B20A206C
:1006D000FFF7E5FFB9FBF0F00A21B0FBF1F201FBF7
:1006E0001208BAF1000F13D1681EA04210DDB8F154
:1006F000000F0BD1B34606EBDB71491001FB04710F
:10070000C8B220220199FFF795FF0FE04FF0010AD0
:10071000B34606EBDB71491001FB0471C8B208F166
:100720003001CAB20199FFF785FF00BF601CC4B257
:10073000AC42C9DBBDE8FF9F2DE9F04104460F46FE
:10074000154600260EE0AA5D39462046FFF772FFE7
:1007500004F10800C4B2782C02DD0024B81CC7B232
:10076000701CC6B2A85D0028EDD1BDE8F0812DE96E
:10077000F04180460E461546002731464046FFF7B9
:1007800005FF00240AE0694A02EB8511085D01219A
:10079000FFF7C6FE781CC7B2601CC4B2102CF2DB97
:1007A000701CC1B24046FFF7F1FE00240CE0690066
:1007B000491C5E4A02EB4111085D0121FFF7B0FEC2
:1007C000781CC7B2601CC4B2102CF0DBBDE8F0810D
:1007D0002DE9F05F06460F4690461C46DDF828A03E
:1007E0004FF0000BE11704EB5171C910A4EBC101EC
:1007F00031B92046E11704EB5171C1F3C70506E09A
:100800002046E11704EB5171C910491CCDB23D4699
:1008100015E029463046FFF7B9FEB1460BE05946D0
:100820000BF1010B1AF801000121FFF779FE09F124
:10083000010000F0FF09C145F1DB681CC5B2A5420B
:10084000E7DBBDE8F09F08B501214FF4967000F09A
:1008500087FDF020ADF8000010208DF80300032084
:100860008DF8020069462F4800F0BEFAF0212D48AD
:1008700000F067FB2020ADF8000069462C4800F02E
:10088000B3FA20212A4800F05CFB0320ADF80000F9
:100890006946274800F0A8FA0321254800F051FBDB
:1008A0004FF40040ADF800006946224800F09CFA81
:1008B0004FF400411F4800F044FB20211C4800F089
:1008C00040FB642000F0CFF82021194800F03BFBEA
:1008D000642000F0C8F82021154800F032FB002108
:1008E000AE20FFF71DFE00210220FFF719FE0021B8
:1008F0001020FFF715FE00214020FFF711FE002118
:100900008120FFF70DFE0021CF20FFF709FE002117
:10091000A120FFF705FE0021C820FFF701FE0021FE
:10092000A62009E000080140C81A000814080020A9
:100930000010014000200140FFF7F2FD0021A82037
:10094000FFF7EEFD00213F20FFF7EAFD0021D32055
:10095000FFF7E6FD00210846FFF7E2FD0021D52064
:10096000FFF7DEFD00218020FFF7DAFD0021D9200E
:10097000FFF7D6FD0021F120FFF7D2FD0021DA209C
:10098000FFF7CEFD00211220FFF7CAFD0021DB207A
:10099000FFF7C6FD00214020FFF7C2FD0021202007
:1009A000FFF7BEFD00210220FFF7BAFD00218D20D8
:1009B000FFF7B6FD00211420FFF7B2FD0021A420AF
:1009C000FFF7AEFD0021A620FFF7AAFD0021AF2012
:1009D000FFF7A6FD0021AF20FFF7A2FDFFF70AFEFB
:1009E00000210846FFF7D2FD08BD000010B56FF0EA
:1009F000040000F07AF92E4800682E49B0FBF1F0AF
:100A00002D4908700846007800EB4001C1EBC0108A
:100A10004FF6FF7101EAC0002849088010BD014669
:100A2000254A12784A434FF0E0235A6100229A6126
:100A30001A46126942F001021A6100BF4FF0E0222B
:100A4000106900F001021AB100F48032002AF5D0DA
:100A50004FF0E022126922F001024FF0E0231A6108
:100A600000229A6170470146144A12884A434FF0A7
:100A7000E0235A6100229A611A46126942F001028B
:100A80001A6100BF4FF0E022106900F001021AB1B4
:100A900000F48032002AF5D04FF0E022126922F0F3
:100AA00001024FF0E0231A6100229A6170470000B2
:100AB0000008002000127A00D4090020D609002086
:100AC00010B54FF4A06000F0C1F810BD014600BFA2
:100AD000704700BF494A128802F04002002AF9D04C
:100AE000C2B2464B1B1D1A80704710B586B0044633
:100AF000012144F2050000F033FC4FF40070ADF822
:100B0000140003208DF8160018208DF8170005A991
:100B10003B4800F069F94FF48060ADF81400042000
:100B20008DF8170005A9364800F05EF925208DF8EC
:100B3000000003208DF801008DF8020001208DF8DF
:100B40000300684600F087F801940020ADF8080023
:100B5000ADF80A00ADF80C00ADF810000C20ADF8AF
:100B60000E0001A9254800F0A2FC012240F2255107
:100B7000224800F034FD0121204800F024FD06B099
:100B800010BD10B540F225511C4800F00DFE10B309
:100B90001A4800F089FDC4B21A48008800F40040E9
:100BA000C8B91848008800F4804060B10A2C03D00E
:100BB00000201449088020E01248008840F40040DA
:100BC0001049088019E00D2C06D10E48008840F429
:100BD00080400C49088010E00A480088C0F30D00EE
:100BE00009490C5407480088401C064908800846FB
:100BF0000088C72801DD0020088010BD00380140B2
:100C000000080140DC090020F40900200948804761
:100C100009480047FEE7FEE7FEE7FEE7FEE7FEE7DE
:100C2000FEE7FEE7FEE7FEE704480549054A064BF6
:100C3000704700001F04000831010008200B00204D
:100C400020110020200D0020200D002031490143FB
:100C5000314A1160704770B5002100230F22C4781B
:100C600004B32D4C246804F4E064C4F5E064210A64
:100C7000C1F10403CA40447804FA03F184781440B3
:100C800021430901254C0678A155047804F01F057D
:100C90000124AC4005786D11AD0005F1E025C5F8E3
:100CA000004109E0047804F01F050124AC401C4D0C
:100CB0000678761145F8264070BD1A4A0A4002436C
:100CC000154B1B1F1A60704739B1134A121D126869
:100CD0000243114B1B1D1A6006E00F4A121D1268D9
:100CE00082430D4B1B1D1A607047042808D14FF03A
:100CF000E021096941F004014FF0E022116107E0B1
:100D00004FF0E021096921F004014FF0E022116168
:100D1000704700000000FA050CED00E000E400E080
:100D200080E100E080FFFF1F10B50446CC488442FC
:100D300008D10121042000F02DFB0021042000F047
:100D400029FB46E0C748844208D10121082000F071
:100D500021FB0021082000F01DFB3AE0C24884423C
:100D600008D10121102000F015FB0021102000F017
:100D700011FB2EE0BD48844208D10121202000F063
:100D800009FB0021202000F005FB22E0B848844246
:100D900008D10121402000F0FDFA0021402000F0A0
:100DA000F9FA16E0B348844208D10121802000F00E
:100DB000F1FA0021802000F0EDFA0AE0AE4884420A
:100DC00007D10121801500F0E5FA0021A01500F0FF
:100DD000E1FA10BD10B50121084600F0DBFA002150
:100DE000012000F0D7FA10BD2DE9F04102460025A0
:100DF0000026002000230024002791F803C00CF0F7
:100E00000F0591F803C00CF0100CBCF1000F03D0DB
:100E100091F802C04CEA050591F800C0BCF1000F42
:100E200031D0146800202BE04FF0010C0CFA00F3D5
:100E3000B1F800C00CEA03069E4220D183004FF0B7
:100E40000F0C0CFA03F7BC4305FA03FC4CEA04044C
:100E500091F803C0BCF1280F06D14FF0010C0CFA39
:100E600000FCC2F814C00AE091F803C0BCF1480FBE
:100E700005D14FF0010C0CFA00FCC2F810C0401C68
:100E80000828D1D31460B1F800C0BCF1FF0F34DDE5
:100E9000546800202EE000F1080C4FF0010808FA19
:100EA0000CF3B1F800C00CEA03069E4221D1830086
:100EB0004FF00F0C0CFA03F7BC4305FA03FC4CEAA5
:100EC000040491F803C0BCF1280F05D100F1080C0F
:100ED00008FA0CF8C2F8148091F803C0BCF1480F6E
:100EE00007D100F1080C4FF0010808FA0CF8C2F81D
:100EF0001080401C0828CED35460BDE8F0814FF626
:100F0000FF710180022181700421C1707047024687
:100F1000002093680B400BB1012000E000207047D7
:100F20000146886880B2704702460020D3680B40B3
:100F30000BB1012000E0002070470146C86880B274
:100F4000704701617047416170470AB1016100E07B
:100F500041617047C16070474FF480320A4382613B
:100F60008161826182698269704702460020434B39
:100F700018684FF68073184040EA021008433F4B50
:100F8000186070473E49C8617047F0B50A460023B3
:100F900000240021002500F00046B6F1004F02D1E8
:100FA000364EF16901E0354E7168C0F3034583B2F6
:100FB00000F44016B6F5401F08D121F070612F4EA5
:100FC000766826F070662D4F7E6012E000F4801681
:100FD000B6F5801F06D1032606FA05F4A14341F0B9
:100FE000706106E0460D360103FA06F6B14341F0A2
:100FF000706122B1460D360103FA06F6314300F066
:101000000046B6F1004F02D11C4EF16101E01B4ECB
:101010007160F0BD30B500228B071C0F0F2303FA5F
:1010200004F2164B08338C1053F824309343134CBE
:1010300008348D1044F8253023468C1053F82430A2
:101040008C07240F00FA04F423430C4C08348D1051
:1010500044F8253030BD0A49DC3108607047000093
:1010600000080140000C0140001001400014014044
:1010700000180140001C0140002001400000014018
:1010800000002042DF48006840F00100DD490860B0
:1010900008464068DC490840DA494860084600686C
:1010A000DA490840D74908600846006820F48020E3
:1010B00008600846406820F4FE0048604FF41F00B6
:1010C00088607047CF49096821F48031CD4A1160AA
:1010D0001146096821F480211160B0F5803F03D0EA
:1010E000B0F5802F0ED106E0C649096841F4803181
:1010F000C44A116007E0C349096841F4A021C14A0C
:10110000116000E000BF00BF704710B5014600222B
:10111000002300204A11012A02D1BA4C236806E0BC
:10112000022A02D1B74C236A01E0B64C636A01F08F
:101130001F02012494401C400CB1012000E000205B
:1011400010BD38B5002000900024002500BF3120DC
:10115000FFF7DBFF05460098401C00900098B0F5B3
:10116000A06F01D0002DF2D03120FFF7CEFF08B1E3
:10117000012400E00024204638BD01460020A14A99
:10118000106820F0F80040EAC10010607047A049E4
:1011900008607047024600209A4B586820F47C1083
:1011A00042EA01031843974B586070479849086614
:1011B000704701460020934A506820F0030008431E
:1011C000506070478F48406800F00C00704701463F
:1011D00000208C4A506820F0F000084350607047AF
:1011E00001460020874A506820F4E06008435060C0
:1011F000704701460020834A506820F4605040EA5E
:10120000C1005060704729B17E4A527A02437D4B3B
:101210005A7204E07B4A527A82437A4B5A72704780
:101220007B49D8310860704701460020754A5068F4
:1012300020F440400843506070470021714A20323A
:101240001170704A82F82010012802D004280AD1B7
:1012500004E001216B4A2032117005E00521694A42
:101260002032117000E000BF00BF7047694908607C
:1012700070476449096A0143624A116270476549CF
:1012800044390860704730B5002100220024002353
:101290005C4D6D6805F00C0121B1042905D00829C9
:1012A00023D105E05C4D056022E05B4D05601FE049
:1012B000544D6D6805F47012524D6D6805F480341C
:1012C000022505EB92421CB9544D554305600BE0D5
:1012D0004C4D6D6805F400351DB1504D554305600A
:1012E00002E04D4D5543056002E04B4D056000BFE7
:1012F00000BF444D6D6805F0F0010909484D6B5C75
:101300000568DD4045603F4D6D6805F4E061090A00
:10131000434D6B5C4568DD4085603A4D6D6805F472
:101320006051C90A3E4D6B5C4568DD40C560354D76
:101330006D6805F44041890B3A4D6B5CC568B5FB9F
:10134000F3F5056130BD29B12E4A526902432D4B98
:101350005A6104E02B4A526982432A4B5A61704712
:1013600029B1284A92690243264B9A6104E0254A32
:1013700092698243234B9A61704729B1214AD2690D
:101380000243204BDA6104E01E4AD26982431D4BBE
:10139000DA61704729B11B4AD2680243194BDA60FF
:1013A00004E0184AD2688243164BDA60704729B1CC
:1013B000144A12690243134B1A6104E0114A12697C
:1013C0008243104B1A6170471249403908607047D8
:1013D0000F49C86470470B49C87170470948406A93
:1013E00040F0807007494862704701460020054A76
:1013F00092680A400AB1012000E0002070470149CC
:1014000088727047001002400000FFF8FFFFF6FEF0
:10141000000042428004424200127A0000093D006E
:10142000DE090020EE09002010B50446FB48844286
:1014300009D101218803FFF7ADFF00214FF480405F
:10144000FFF7A8FF32E0F648844209D101214804A1
:10145000FFF7ADFF00214FF40030FFF7A8FF25E0B4
:10146000F048844209D101218804FFF7A0FF002140
:101470004FF48020FFF79BFF18E0EB48844209D12E
:101480000121C804FFF793FF00214FF40020FFF76C
:101490008EFF0BE0E548844208D101210805FFF7E3
:1014A00086FF00214FF48010FFF781FF10BD2DE96A
:1014B000F04786B005460E460024A24600BFA1466E
:1014C0000027B08900B100BF2F462C8A4CF6FF7070
:1014D0000440F08804432C82AC894EF6F31004409B
:1014E000B08831890843718908430443AC81AC8AD0
:1014F0004FF6FF400440B0890443AC8201A8FFF7D7
:10150000C2FEC648874202D1DDF810A001E0DDF836
:101510000CA0A88900F4004040B10AEBCA0000EB1F
:101520000A1031684900B0FBF1F807E00AEBCA0085
:1015300000EB0A1031688900B0FBF1F86420B8FBB9
:10154000F0F004012009642101FB1089A88900F44E
:10155000004040B1322000EBC900B0FBF1F000F0D8
:101560000700044308E0322000EB09106421B0FBBF
:10157000F1F000F00F0004432C8106B0BDE8F087C5
:101580004FF41651016000218180C18001810C213E
:10159000418100218181704710B502460020108AE8
:1015A0004FF2FF0318400B884C8823438C88234359
:1015B000CC8823431843108210BD00210180418054
:1015C0008180C180704721B1828942F400528281BA
:1015D00004E082894DF6FF731A4082817047F0B5AE
:1015E0000346002400260025002040F66A17B94271
:1015F00000D100BF1846C1F3421401F01F060127B5
:1016000007FA06F5012C01D10C3004E0022C01D1BF
:10161000103000E014301AB107682F43076002E071
:101620000768AF430760F0BD1AB1838A0B4383821A
:1016300002E0838A8B4383827047028A4FF6F073FD
:101640001A400282028A0A430282704782894FF25C
:10165000FF731A40828182890A438281704721B1D7
:10166000828942F00202828104E082894FF6FD7392
:101670001A4082817047028A4FF6DF731A40028255
:10168000028A0A430282704721B1028A42F48042F0
:10169000028204E0028A4BF6FF731A40028270470E
:1016A000C1F308028280704701468888C0F30800B1
:1016B0007047818941F0010181817047028BD2B26C
:1016C0000283028B42EA012202837047028B02F4FA
:1016D0007F420283028B0A430283704721B1828AD0
:1016E00042F02002828204E0828A4FF6DF731A40C1
:1016F0008282704721B1828A42F01002828204E025
:10170000828A4FF6EF731A408282704721B1828A33
:1017100042F00802828204E0828A4FF6F7731A4090
:101720008282704721B1828942F40042828103E0C3
:101730008289C2F30E028281704721B1828A42F40B
:101740000062828204E0828A4FF2FF731A40828232
:101750007047828A4FF6FB731A408282828A0A435C
:101760008282704721B1828A42F00202828204E0C2
:10177000828A4FF6FD731A4082827047024600202B
:10178000B1F5007F00D100BF13880B400BB10120E1
:1017900000E00020704701F40072B2F5007F00D134
:1017A00000BFCA430280704770B502460024002380
:1017B0000025002040F66A16B14200D100BFC1F3F7
:1017C000421501F01F03012606FA03F3012D02D191
:1017D0009689334006E0022D02D1168A334001E09B
:1017E000968A33400C12012606FA04F41688344017
:1017F00013B10CB1012000E0002070BD10B5002233
:10180000002340F66A14A14200D100BF0A1201244D
:101810009440A3B2DC43048010BD000000380140B6
:101820000044004000480040004C00400050004090
:1018300070477047704770477047754600F02CF846
:10184000AE4605006946534620F00700854618B0AD
:1018500020B5FFF7E9F9BDE820404FF000064FF052
:1018600000074FF000084FF0000B21F00701AC46D5
:10187000ACE8C009ACE8C009ACE8C009ACE8C009F4
:101880008D46704710B50446AFF300802046BDE892
:101890001040FEF7B8BC000000487047BC0A0020AA
:1018A0000000000000000000002F00000000070002
:1018B000070000147F147F1400242A7F2A1200627C
:1018C0006408132300364955225000000503000028
:1018D00000001C224100000041221C000014083EB0
:1018E00008140008083E0808000000A06000000876
:1018F00008080808000060600000002010080402CA
:10190000003E5149453E0000427F40000042615187
:101910004946002141454B31001814127F10002721
:1019200045454539003C4A494930000171090503E4
:1019300000364949493600064949291E0000363615
:101940000000000056360000000814224100001478
:101950001414141400004122140800020151090655
:1019600000324959513E007C1211127C007F4949D6
:101970004936003E41414122007F4141221C007F07
:1019800049494941007F09090901003E4149497A15
:10199000007F0808087F0000417F4100002040418F
:1019A0003F01007F08142241007F40404040007FFB
:1019B000020C027F007F0408107F003E4141413E3F
:1019C000007F09090906003E4151215E007F091987
:1019D00029460046494949310001017F0101003F84
:1019E0004040403F001F2040201F003F4038403F04
:1019F0000063140814630007087008070061514968
:101A0000454300007F41410000552A552A550000FA
:101A100041417F0000040201020400404040404078
:101A2000000001020400002054545478007F484410
:101A3000443800384444442000384444487F003847
:101A40005454541800087E0901020018A4A4A47C70
:101A5000007F080404780000447D4000004080843A
:101A60007D00007F102844000000417F4000007C82
:101A700004180478007C080404780038444444388E
:101A800000FC242424180018242418FC007C0804DA
:101A9000040800485454542000043F444020003CB3
:101AA0004040207C001C2040201C003C4030403C3A
:101AB000004428102844001CA0A0A07C00446454CA
:101AC0004C4414141414141400000000000000000E
:101AD0000000000000000000000000F8000000000E
:101AE000000000333000000000100C06100C06004F
:101AF000000000000000000040C07840C0784000B6
:101B0000043F04043F040400007088FC0830000017
:101B1000001820FF211E0000F008F000E01800006F
:101B200000211C031E211E0000F008887000000028
:101B30001E2123241927211010160E00000000007A
:101B40000000000000000000000000E01804020097
:101B5000000000071820400000020418E000000008
:101B60000040201807000000404080F08040400006
:101B70000202010F01020200000000F0000000005C
:101B80000101011F01010100000000000000000030
:101B900080B07000000000000000000000000000A5
:101BA000000101010101010100000000000000002E
:101BB00000303000000000000000000080601804C9
:101BC000006018060100000000E010080810E000A6
:101BD000000F102020100F00001010F8000000006F
:101BE0000020203F202000000070080808887000B6
:101BF0000030282422213000003008888848300036
:101C00000018202020110E000000C02010F8000055
:101C100000070424243F240000F8088888080800EE
:101C20000019212020110E0000E010888818000003
:101C3000000F112020110E0000380808C8380800D5
:101C40000000003F00000000007088080888700055
:101C5000001C222121221C0000E010080810E000D6
:101C60000000312222110F00000000C0C00000005F
:101C70000000003030000000000000800000000084
:101C8000000080600000000000008040201008007C
:101C90000001020408102000404040404040400045
:101CA0000404040404040400000810204080000020
:101CB0000020100804020100007048080808F00025
:101CC0000000003036010000C030C828E810E000F5
:101CD0000718272423140B000000C038E000000080
:101CE000203C23020227382008F8888888700000EA
:101CF000203F202020110E00C030080808083800BE
:101D0000071820202010080008F808080810E00034
:101D1000203F202020100F0008F88888E8081000D5
:101D2000203F20202320180008F88888E8081000A9
:101D3000203F200003000000C030080808380000E1
:101D400007182020221E020008F808000008F808E2
:101D5000203F210101213F20000808F80808000069
:101D60000020203F2020000000000808F80808009C
:101D7000C08080807F00000008F888C02818080014
:101D8000203F20012638200008F80800000000004D
:101D9000203F20202020300008F8F800F8F8080044
:101DA000203F003F003F200008F830C00008F8083E
:101DB000203F200007183F00E01008080810E0004E
:101DC0000F10202020100F0008F808080808F00065
:101DD000203F210101010000E01008080810E00088
:101DE0000F18242438504F0008F88888888870001D
:101DF000203F2000030C30200070880808083800BD
:101E00000038202121221C00180808F808081800B2
:101E10000000203F2000000008F808000008F80833
:101E2000001F202020201F000878880000C83808E4
:101E3000000007380E010000F80800F80008F8005C
:101E4000033C0700073C03000818688080681808F6
:101E500020302C03032C30200838C800C838080074
:101E60000000203F2000000010080808C8380800C3
:101E70002038262120201800000000FE0202020067
:101E80000000007F40404000000C30C00000000017
:101E9000000000010638C00000020202FE0000003F
:101EA000004040407F0000000000040202020400E5
:101EB0000000000000000000000000000000000022
:101EC000808080808080808000020204000000000A
:101ED0000000000000000000000080808080000002
:101EE0000019242222223F2008F8008080000000F0
:101EF000003F112020110E000000008080800000B3
:101F0000000E112020201100000000808088F800C1
:101F1000000E112020103F200000808080800000F3
:101F2000001F222222221300008080F08888881857
:101F30000020203F20200000000080808080800062
:101F4000006B94949493600008F8008080800000F7
:101F5000203F210000203F200080989800000000D2
:101F60000020203F20200000000000809898000002
:101F700000C08080807F000008F800008080800022
:101F8000203F24022D302000000808F80000000047
:101F90000020203F20200000808080808080800002
:101FA000203F20003F20003F808000808080000094
:101FB000203F210000203F20000080808080000022
:101FC000001F202020201F00808000808000000053
:101FD00080FFA12020110E00000000808080800082
:101FE000000E112020A0FF80808080008080800073
:101FF00020203F21200001000000808080808000A0
:102000000033242424241900008080E08080000014
:102010000000001F20200000808000000080800061
:10202000001F202020103F208080800000808080C2
:1020300000010E3008060100808000800080808052
:102040000F300C030C300F00008080008080800077
:102050000020312E0E3120008080800000808080A2
:1020600080818E7018060100008080808080800052
:102070000021302C2221300000000000807C020270
:1020800000000000003F404000000000FF00000092
:1020900000000000FF0000000002027C8000000041
:1020A0000040403F0000000000060101020204045D
:1020B0000000000000000000D82000080000002000
:1020C000F40900006C0100089C230008F4090020BA
:1020D0002C070000D001000840120003050911FF81
:1020E000118905C300E000F000F8000100083A443F
:1020F00028FF11AA440001500B83013844829292B8
:102100007401831120087C44FF017D7D7D0441051D
:1021100040047D01FF6E920102613F033B01017E9D
:1021200081419149F20101011BC230083F3F030385
:10213000F3131101100601F1116181402005816145
:1021400011F14733414107200401C12120A321C1DE
:102150001431193137040736D33303033F3F42604C
:1021600006E0E000007FA8127FBF40040618060AC0
:102170001008000040407F4040A410041F20400190
:10218000A3201F143300600E6004300C0346053496
:10219000C21004070706017009040404844444447F
:1021A000840780050484C4041501120A71112140BA
:1021B000073D0707C9200F00001018141211000076
:1021C0000F1010100F0F131F1015600D08101212B2
:1021D0000D00001800000D120A51295130015E0156
:1021E000528001013B4514047F030CA915DE1C0538
:1021F000385454582503080A2004047800003C4051
:10220000407C2000092CFFAAAAAA280800FF681019
:10221000062649494932101005020408100F0D6FB7
:1022200000049D01040D9D0004156343F80801247A
:102230000500F81860E8240480601823572020293E
:1022400023E01021A310E01449B4313908043C887C
:102250006818630D15FF037DEA039DFF0371144D9C
:10226000FF031D06043D2E040942E91C0640202000
:1022700020C04A04110721EA3E40520452600E81F8
:1022800018712951070D4769031C060C0A0A090C2D
:102290000004156B2D00042004080F081510050814
:1022A00009090E071D180430050909090F0A5129EB
:1022B00051070DFF00040D2200047C04A24A041FF4
:1022C000071C0B020304060708090000F06A052337
:1022D00010FF050E13F091052E0FED052EFF0606DB
:1022E0000A120F2F100840405F55555575045B5F6B
:1022F0004094D95024060F09498979B70211201F4B
:10230000200800FE02424ACA4A030C04124202FE9E
:10231000F904000C1340504C4340404F50505C4077
:10232000FE13F8880122FF050E13F8DA072E1F9D11
:1023300003227F2003109F80E2338082010C071666
:10234000E2A2928A8682DF050C041640807F38085C
:10235000040B142424A4FEA3220022CC009C1F08FA
:1023600006F9083E0131070C0510FF020202EF06D4
:10237000257C539008C3FE0898070C0F1E04448266
:102380007F01808040432C102846817F0625D6653A
:0C239000DA00070002040608000000004C
:0400000508000131BD
:00000001FF
